:100000005E28000008000120900B0328080005303E
:100010008D0006308C008C0B0B288D0B09280800F6
:100020000720910B102808002F0889002E0888004F
:1000300083168B1355308900AA30890088146430E8
:10004000910010202F0889008316081483120808D5
:10005000AE000800051A35280518970A8518970B71
:100060000519960A8519960B3A280518950A8518D8
:10007000950B3A281508AE00AF0001301420160881
:10008000AE00AF00023014201708AE00AF000330FE
:10009000142004308C000000FF30910010208C0BE5
:1000A0004B280800143095008A009600AE000530F9
:1000B0009700AE00283098002A208428FF30860060
:1000C000003066001F306500051A52280130AF006D
:1000D00022202E0895000230AF0022202E08960024
:1000E0000330AF0022202E08970028309800842883
:1000F0000610150890000320061408008611170842
:100100009000032086150800782016089000032030
:100110007E2018089100102005182A2085182A2012
:0A01200005192A2085192A208428D9
:00000001FF
